:020000040000FA
:100000003E2D203420342034203420342034003459
:100010004C346F3463346B34653464340034593495
:100020006534733400344E346F34003453346534E3
:100030007434753470343F340034543469346D345E
:1000400065340034503472346F3467347234613440
:100050006D34003443346C34723400344E347834AC
:10006000743400340D342334203400340D343F34E0
:1000700020340034433448342034503472346F34E4
:100080006734723461346D346D34653472340034E5
:100090000D340034563432342E3430342E3432346D
:1000A0002034323438342F34303435342F34303433
:1000B000353400344534723400344D346F340034F8
:1000C000543475340034573465340034543468344F
:1000D00000344634723400345334613400345334C1
:1000E000753400344F346E342034003420344F34AF
:1000F0006E3400344F346634663400340D34433487
:100100002F34483465346134743469346E34673460
:100110003A34203400340D3448346F34743420348D
:10012000573461347434653472343A3420340034D2
:1001300049343234433420344534723400340D347D
:10014000543469346D346534203400340D344D3406
:1001500065346D346F347234793420340034523461
:1001600054344334203469346E3469347434003484
:1001700052345434433420344F346B3400342034FC
:100180005734653465346B3420340034203477348C
:100190002F344534203420340034203441346C343E
:1001A0006C34203420340034663472346534653461
:1001B00000342C342034503472346F346734723449
:1001C00061346D3400342C3420344D3461346E3459
:1001D000753461346C3400344D3461346E34003421
:1001E0005034723467340034573444345434203437
:1001F00000341B346334003400348A012108820047
:10020000A100FD2000380319080055210D3A0A30DD
:1002100003195521A10A012948300029A100FD2018
:10022000003803190800CF21A10A0F2963212308F0
:1002300055212208552963212308CF212208CF29DF
:10024000AF00A6302329FF3E031D2229AF03031D63
:1002500021290800C90108302021B427C903031D42
:100260002B29B42FC90113302021B427C903031D42
:10027000332901308A003208B300B201C9014908AC
:100280004E218500003E03194A29B20D051E321485
:10029000C90A3F293208B306B305B42F82073F3499
:1002A00077347B347D347E3400340C1E552999001C
:1002B00008008C1E59291A0818196029981C080072
:1002C00018121816FF34A40069212308A200A40EF6
:1002D00069290F302405F63E0318073E3A3EA30075
:1002E0000800A601A200463C031C872941302202D7
:1002F000031C7D290A3EA40008002208393C031C87
:10030000872930302202031C8729A4000800A60A8E
:10031000080022087121A608031D0800240EA5006C
:1003200023087121A608031D08002408A504A50EB2
:1003300008000430E721F10104302322A121AD217E
:10034000080008307A020318FA0101308A007A089E
:10035000B6210E212030CF2108007908C921771C51
:10036000EF217718F1217808C921080082075A3453
:100370005D3460346334663469346C346F34B00097
:10038000300E0F398500DF2130080F398500DF215D
:10039000DA29B100310ECD2131080F393038B000E3
:1003A000300E0F3940388500DF2130080F394038D2
:1003B0008500DF210A30FF3E031DDB290800851779
:1003C0000000851308008030BF29C030BF29803E5F
:1003D000BF29C03EBF290D30BF290C30BF293A309C
:1003E000CF292030CF295E30CF290130BF21023004
:1003F00020292030BF212830BF210630BF210C30FA
:10040000BF21F529E3210822E329E5210822E52976
:100410001030C900F121C90B0A2A08008316F20026
:100420003B2286227008FE394122F4180800710828
:100430004122F418080072084122F41808008E22A4
:100440008312740808008316F6003B228622700887
:10045000FE394122F418080071084122F4180800FE
:100460008622700801384122F418080066228E2284
:1004700000088312080083120608F63986008316E6
:1004800008008316F3000830F5008422F30D031CE6
:100490000610031806148122F503031D462A0614CC
:1004A000F40186158312061C622A8316F50B522A64
:1004B000F4148E22831248300021983000214830F5
:1004C00000210800831684228611080077308400FA
:1004D00006140830F5000310800D8615842283125F
:1004E0000608831686110139031D0014F50B6B2ACB
:1004F000F60B7D2A06148122080006108122840A48
:10050000682A8615842286110000080006148615C4
:100510008422061084228611842208008611061087
:1005200084228615842206140800D030F0000030A2
:10053000F100043023227908C6007808C5007A0843
:10054000C70048084506031908000730F1000A30C3
:10055000C90004302322B4220330F107C903031D6C
:10056000A92A4508C800080078084506031D0800A8
:1005700079084606031D0800FA08031908007A19CD
:10058000CD2AFA18C82A47080A3E831CCD2A08003B
:1005900047080A3E8318CD2A0800281BD52A7A1E50
:1005A000D52A7A1B27177A1F2713A81B0800FA1EC3
:1005B0000800FA1BA717FA1FA7130800840A0008EF
:1005C000203A031DAD2E840A00087121FA00840A26
:1005D0000008203A031DAD2E0C232618AD2EF9007D
:1005E000DC3E0318AD2E840A00083A3A031DAD2EF6
:1005F0000C232618AD2EF800A03E0318AD2EF101F5
:1006000003010E22F10A78080E22F10A79080E225F
:10061000F10A7A080E220800840A0008A300840A5E
:100620000008A200892125080800840A000803198F
:10063000842B71212618AD2E063E8318AD2EFA3E6E
:100640000310F100240D7107083EF100840A000830
:10065000203A0319332B0008783A031DAD2EF80118
:10066000F901FA015A2BFA01840A00080319AD2E88
:10067000203A03193D2B6323342BF0307A050319FC
:10068000AD2E0F307A050319AD2E0C23F900261874
:10069000AD2EDC3E0318AD2E840A00083A3A031D45
:1006A000AD2E0C23F8002618AD2EA03E0318AD2E5B
:1006B0000C21A52378080E22F10A79080E22F10AEE
:1006C0007A080E2208000008633A03197A16000817
:1006D000433A031D6D2B7A177A160008683A0319FE
:1006E000FA160008483A031D772BFA17FA166130FC
:1006F000000603197A15653000060319FA147730DD
:10070000000603197A140800C9010730F1004830C7
:100710000021703055214908303E552120305521A7
:10072000043023227A08031D982BD4300021992B02
:10073000A523483000210330F107C90A0A304906D1
:10074000031D892B4830002108002D30FA1A68302B
:10075000FA1B483055212D307A1A63307A1B43300A
:100760005521BF30FA18C6307A19CD3000217908EA
:1007700016213A3055217808162108003318CE2B5F
:10078000B318CB2B3319D42BB319D12B331E08003C
:10079000D723F52108004030A70608008030A706BF
:1007A00008004030A80608008030A8060800F5219F
:1007B0000230E72116300E210D30E7210F300E21D7
:1007C0000E30E92113300E21AC01AC0303190800EF
:1007D000193020213921B2180800B21DE52B0C3048
:1007E000E7211D300E210930E92122300E2132246B
:1007F000B218832CB21DF72BF52138244124D030B8
:10080000F0000030F10004302322F70106307C2490
:100810000630E721A1210930AD2132243218162CEF
:10082000B219FA0AB218FA032B24062C1924FF2253
:1008300008000630792409307C2479308400DC30CB
:10084000AA004D24093079240C307C248403A03084
:10085000AA004D2408007A0803190730FA1901305C
:10086000FA0008000F30202139210319322C08002A
:100870000F30E7212B30CF210F30E9212D30CF2150
:100880000800E5212E300E210800E3212A300E2138
:100890000800E521F0300E2108000930E721AD21E4
:1008A000322432180800B218612CB21D4D2C0008F9
:1008B000073E831CFA3E80002A08000703188001C7
:1008C0004D2C01300002831CF939800003184D2C97
:1008D00059308000A0302A0603194D2C23308000A7
:1008E0004D2C0003063E831CF93E03182A098000A4
:1008F0004D2CE921F121F129E921F321F329E92105
:10090000F129E921F329AB01F521382445244924B3
:100910000730E9215030CF210830E9212B08CD21C3
:100920002B08AC24BD243224321A0800B2199F24AB
:10093000B218A6243218E12C3219DD24862CF730A7
:100940002B070319AB01031DAB0A08000A30AB08E3
:100950000319AB00AB030800B524F10304302322D4
:10096000F7010800B5245A23080003102B08F100F2
:100970002B0D7107083EF10008007A08031DC62CF4
:1009800035250430E721D4300E2108000430E7215A
:100990002D30FA1A6830FA1B4830CF212D307A1AE0
:1009A00063307A1B4330CF21F1217730FA1865305C
:1009B0007A196130CF21F121AD29F801F901FA014D
:1009C000B22C4124FA1607307924E321F121F121D8
:1009D000F12104307C24AC010830AD00BD24322468
:1009E0003218FC2CB2191525B2181B2529250F30F9
:1009F000FA052925FA04EE2C0430792407308124E5
:100A0000AC010330AD00BD2432243218102DB219D0
:100A10001525B2181B25F030FA052225FA04032DFE
:100A200019240C307924B224862CAC0A2D082C060B
:100A30000319AC010800AC08031D202D2D08AC00E3
:100A4000AC03080005308A002C0882070134023408
:100A5000043405308A002C0882072034A034103476
:100A600050343034B0347034F0340A30CA000430BA
:100A7000E721F121CA03031D392D08008313073034
:100A80009F008501860183169F01303085003B3031
:100A900086008117011501158115181218151930D6
:100AA000990098168E22831298171816031A632D30
:100AB00099302E06031D2E0A063E831CFA3EAE0018
:100AC0000319AE0A642DAE01C8302021F93000218F
:100AD000F9213A300E21B20105224A300E212A2195
:100AE000052239272A21F5213D30F100013023224A
:100AF000A700F10301302322A800F10301302322D3
:100B0000A9003530B400FF30C8003A30002132303F
:100B10000021992195223921291CBE230F30CB00B9
:100B2000013020218C1AE225CB0B902D9825892DA0
:100B300083120530E9210130291808300E212E08D2
:100B40000319A82D0530E921F4300E212E08C92102
:100B500074080319AF2D0530E92198300E210030BB
:100B6000E721EC30A81FF0300E210D30E721EC30EA
:100B7000281FF0300E21271FCE25271BD325A71FA6
:100B8000D825A71BDD253B30F10029080E22F10AEC
:100B900028080E22F10A27080E22080006130D303D
:100BA000E9217A300E2906170D30E92176300E2919
:100BB00086130030E9217A300E2986170030E921AA
:100BC00072300E29CB01CB0A3408840059218000F1
:100BD000FF3A0319080000080D3A0319002E000817
:100BE0005521840A0408453A0319F92D0408B40074
:100BF0000800363000213530B400323000210800C2
:100C000080010326FB2D353084000008031D092ECA
:100C10000800763000060319B42E7530000603195B
:100C2000C52E6D3000060319DE2E6F300006031945
:100C3000F72E6430000603190C2F733000060319D9
:100C4000DE2A703000060319152B743000060319D4
:100C50001F2F663000060319B82E56300006031900
:100C6000B02E723000060319572E77300006031994
:100C70008B2E5230000603193E2D713000060319E9
:100C80004A2E5130000603194D2E48300006031934
:100C9000472EAD2EF10157300E2AF1015730F700E3
:100CA0005930F8002130F9000130FA00FF2A840A97
:100CB0000008203A031DAD2E840A0008A300840A10
:100CC0000008A20089212618AD2E2508F100840A0B
:100CD0000008203A031DAD2E840A0008A300840AF0
:100CE0000008A20089212618AD2E25080319013E0F
:100CF000CA00F73E0318AD2EA63000214A08232271
:100D0000773084000008162120305521840ACA0358
:100D1000031D822E0C29840A0008203A031DAD2EE3
:100D2000840A0008A300840A0008A200892126186A
:100D3000AD2E2508F100840A0008203A031DAD2ECF
:100D4000840A0008A300840A0008A200892126184A
:100D5000AD2E25080E220C29312E36300021080038
:100D6000F9300021503020290C214A3000210800A0
:100D7000840A65300006031DBF2E29100800643068
:100D80000006031DAD2E29140800840A63300006F6
:100D9000031DCC2E2713080043300006031DD22E5E
:100DA0002717080068300006031DD82EA713080077
:100DB00048300006031DAD2EA7170800840A6330D3
:100DC0000006031DE52E2813080043300006031D0E
:100DD000EB2E2817080068300006031DF12EA8131B
:100DE000080048300006031DAD2EA81708007E300D
:100DF00000217A30271B76300021D930281BE330C0
:100E000000218B3000217A30A71B76300021D930A9
:100E1000A81BE330002108000C21840A773000066B
:100E200003191D2F73300006031DAD2E270E0C393C
:100E3000A4002808C039240416292E0816299F303A
:100E40000021D030F0000030F100043023220130C6
:100E50008A007A08B6210021203055217908162110
:100E60003A305521780816213A3055217708162155
:100E70000800D030F000F10101302322F71B4D2F84
:100E80003E30F10002302322423A031D4D2F7708F5
:100E9000BB3A031D4D2FB8300E29D030F000003082
:100EA000F1000E220730F10000300E220830F10070
:100EB0003630CA0003010E22F10ACA0B5A2F3E3007
:100EC000F100BB300E22F10A42300E220130FA004E
:100ED000F901F801FF22AF300E2132295034493494
:100EE00043342034483465346134743469346E34A6
:100EF00067342034503472346F3467347234613460
:100F00006D346D346534723420342F3420344334DE
:100F10006F346E34743472346F346C346C346534C2
:100F2000723443346F3470347934723469346734D2
:100F3000683474342034283443342934203432342F
:100F40003034303435342E342034503465347434F5
:100F5000653472342034473472346934663466340C
:0C0F600069347434683473346400080091
:02400E00143F5D
:00000001FF
